:10000000FAC014C113C112C111C110C10FC10EC178
:100010000DC10CC10BC10AC109C108C107C106C18C
:1000200005C104C120C147C101C100C1FFC0FEC05C
:10003000FDC0FCC02B4154455849540D0A002B4FBC
:100040004B0D0A002B61746174002B415441540024
:100050002B4F4B0D0A004552520D0A0041542B42C2
:100060004C0041542B5354520041542B474F544F92
:100070000041542B434C520041542B424155440003
:1000800041542B4543484F0044656275674469738A
:10009000706C61792076312E302028486F62626959
:1000A000656C656B74726F6E696B612E68752C2060
:1000B000627920546F7069290D0A0041542B56450E
:1000C000523F0041542B424C205B302D3235355D80
:1000D000202D2053657420646973706C61792062EF
:1000E00061636B6C69676874206272696768746EBB
:1000F0006573730D0A0041542B535452207374726C
:10010000202D205072696E7420737472696E670DB1
:100110000A0041542B474F544F20782079202D203E
:10012000476F746F2058590D0A0041542B434C52AD
:10013000202D20436C65617220646973706C617955
:100140000D0A0041542B42415544205B302D335D54
:100150002053657420626175647261746520283073
:100160003D393630302C20313D31393230302C2081
:10017000323D35373630302C20333D313135323059
:1001800030290D0A0041542B4543484F205B302F46
:10019000315D202D204563686F206F66662F6F6E7E
:1001A0000D0A0041542B5645523F202D20446973BF
:1001B000706C6179206E616D6520616E642076657A
:1001C0007273696F6E20696E666F0D0A000D0A2DDD
:1001D0002D2D2D2D2D2D2D2D2D2D2D2D2D2D2D2D4F
:1001E0002D2D2D2D2D2D0D0A003F0041542B48455E
:1001F0004C500041540011241FBECFEFD4E0DEBFAD
:10020000CDBF11E0A0E0B1E0E2EDFAE002C0059060
:100210000D92AC31B107D9F712E0ACE1B1E001C009
:100220001D92A532B107E1F7E7D251C4E9CE9B0197
:10023000AC0160587B47814E9F4FF3E0660F771FFC
:10024000881F991FFA95D1F7E4E0220F331F441F4E
:10025000551FEA95D1F710D4215030402093C400A7
:100260003093C50008951F920F920FB60F9211247C
:100270008F939F93EF93FF938091C0009091C6005E
:100280008C7181F48091A001E82FF0E0E25EFE4FD6
:1002900090838F5F8093A0018091A001803410F043
:1002A0001092A001FF91EF919F918F910F900FBE3F
:1002B0000F901F9018951F920F920FB60F92112456
:1002C0008F939F93EF93FF939091A3018091A1014E
:1002D0009817C1F08091C00080648093C000909115
:1002E000A101E92FF0E0EB55FE4F80818093C6001D
:1002F0009F5F9093A1018091A10187FF08C0109298
:10030000A10105C08091C1008F7D8093C100FF9144
:10031000EF919F918F910F900FBE0F901F901895A6
:100320009091A00180915F01981711F4E0E010C056
:1003300080915F01E82FF0E0E25EFE4FE0818F5F89
:1003400080935F0180915F01803410F010925F0113
:100350008E2F08959091A301E92FF0E0EB55FE4F09
:1003600080839F5F9093A3018091A30187FF02C0C8
:100370001092A3018091C10080628093C100089512
:10038000CF93DF93EC0102C02196E4DF88818823BC
:10039000D9F7DF91CF910895CF93DF93EC01FE0160
:1003A0008491882319F0D6DF2196F9CFDF91CF9180
:1003B00008951F93182F64E63FD3805DCBDF812F14
:1003C00064E63AD3192F892F6AE036D3805DC2DF05
:1003D000812F6AE031D3892F805DBCDF1F910895A2
:1003E0009091A3018091A1019817D1F70895519A96
:1003F000509888E98093C10086E08093C200809184
:10040000C6008091C00087FDFACF80EC8093C000C9
:100410008091C6001092A00110925F011092A40179
:100420001092A3011092A10160E875E280E090E0D3
:10043000FEDE089520E43CE904C0F9013197F1F7AC
:1004400081508823D1F70895FC0120E03AE00DC0E7
:100450009D3071F09A3061F0903251F0239F802DE1
:100460001124292F2053280F31969081992381F749
:10047000822F08951F93182F64E6DED2805D6ADF15
:10048000812F64E6D9D2192F892F6AE0D5D2805DF9
:1004900061DF812F6AE0D0D2892F805D5BDF1F9101
:1004A0000895EF92FF920F931F93DF93CF93CDB7F1
:1004B000DEB728970FB6F894DEBF0FBECDBF809190
:1004C0006001882309F40BC1FE013196CE01099623
:1004D0001192E817F907E1F700E611E020E030E0BB
:1004E000BE016F5F7F4F422FF80191918F01892FDD
:1004F00081568A3108F49052992379F0903269F04C
:100500009D3359F0FB01E20FF31F90834F5F2F5F84
:100510003F4FF1E007361F0731F7FE01E40FF11DF1
:100520001182F8018081803211F08D3311F40F5F58
:100530001F4F7E010894E11CF11CC70163EF71E0BD
:10054000BDD2892B09F4C8C0C7016BEE71E0B6D2E9
:10055000892B39F0C70169EE71E0B0D2892B09F01F
:1005600049C08DEC91E018DF9091A3018091A10129
:100570009817D1F783EA91E00FDF9091A301809162
:10058000A1019817D1F785E891E006DF9091A301CA
:100590008091A1019817D1F783E491E0FDDE90915D
:1005A000A3018091A1019817D1F78AE291E0F4DECE
:1005B0009091A3018091A1019817D1F782E191E078
:1005C000EBDE9091A3018091A1019817D1F786EFFE
:1005D00090E0E2DE9091A3018091A1019817D1F7FC
:1005E00083EC90E0D9DE9091A3018091A10198174E
:1005F000D1F772C0C7016BEB70E060D2892B19F4A0
:1006000088E890E068C0C70160E870E057D2892BA5
:1006100059F4C80119DF10921C01813309F05CC044
:1006200081E080931C0158C0C70168E770E046D2A2
:10063000892BE9F4C80108DF823049F0833061F08A
:10064000813079F460E07BE480E090E00EC060E00F
:1006500071EE80E090E009C060E072EC81E090E033
:1006600004C060E875E280E090E0E1DD35C0C701DC
:1006700061E770E023D2892B11F479D12DC0C70135
:1006800069E670E01BD2892B81F4C801DDDEF82E0B
:1006900001C08F01F801819180538A30D0F3CF01DE
:1006A000D3DE682F8F2D59D117C0C70162E670E0E5
:1006B00005D2892B19F4C80172D10EC0C7016CE5AF
:1006C00070E0FCD1892B29F4C801BEDE8093B40010
:1006D00003C086E590E060DE80E590E05DDE289670
:1006E0000FB6F894DEBF0FBECDBFCF91DF911F9143
:1006F0000F91FF90EF9008951F939091A00180912A
:100700005F01981709F45CC00BDE182F80911C0163
:10071000882311F0812F1EDE1D3061F580E691E007
:100720006AE470E0CBD1892B39F080E691E064E493
:1007300070E0C4D1892B41F48EE390E02DDE81E09E
:1007400080931D011092600180911D01882361F446
:100750006091A20102D180E691E021D18091A201B5
:100760008F5F8093A20101C09CDE10925E01109207
:10077000600126C01B3189F4FAD0109260011092FA
:100780005E011092A20180911D018823C9F084E3CB
:1007900090E002DE10921D0113C0103288F08091AB
:1007A0005E018F3368F4E82FF0E0E05AFE4F1083CB
:1007B000E82FEF5FE0935E01F0E0E05AFE4F108219
:1007C0001F910895539A13DE83E28093B00084E072
:1007D0008093B10088EC8093B4008CE0F8D0C7D04F
:1007E000C6D0789481E080931C0110925E01109233
:1007F000A20110921D010895E5DF80E060E0ADD018
:1008000080E091E0CCD080E061E0A7D080E191E091
:10081000C6D022E340E45CE903C0CA010197F1F7C6
:100820002150D8F769DFFECF662311F02A9A01C064
:100830002A982998549A559A569A579A5F985E988A
:100840005D985C9887FD5F9A86FD5E9A85FD5D9A4E
:1008500084FD5C9A289A00C028985F985E985D98FD
:100860005C9883FD5F9A82FD5E9A81FD5D9A80FDB2
:100870005C9A289A00C028985C9A5D9A5E9A5F9A62
:100880000895882311F02A9A01C02A98299A549829
:10089000559856985798289A00C04C9B02C080E102
:1008A00001C080E04D9980624E9980644F998068C4
:1008B000289800C0289A00C04C9981604D998260A8
:1008C0004E9984604F9988602898089580E0D9DF18
:1008D00087FDFCCF88E090E00197F1F780E0D1DF61
:1008E00008951F93182FF2DF812F60E09DDF1F9185
:1008F00008951F93182FEADF812F61E095DF1F9184
:1009000008950F931F938C0168EE73E0A1D0862F9A
:10091000805DEFDFC80168EE73E09AD0182F092FD1
:1009200064E670E095D0862F805DE3DF812F902F05
:1009300064E670E08DD0182F092F6AE070E088D04F
:10094000862F805DD6DF812F902F6AE070E080D007
:10095000805DCFDF1F910F910895662311F48058B9
:1009600001C08054BEDF0895B1DF90E0089581E0BA
:10097000B8DF089582E0B5DF08951F93182FA6DF32
:100980001A3041F4803410F080E001C080E48058D7
:10099000A8DF03C0812F61E047DF1F910895CF9347
:1009A000DF93EC0101C0E9DF89918823E1F7DF9152
:1009B000CF910895CF93DF93EC0101C0DEDFFE01FC
:1009C000219684918823D1F7DF91CF9108951F93C9
:1009D000182F229A219A209A549A559A569A579AE1
:1009E00080E09AEF0197F1F75D9A5C9A289A00C02F
:1009F000289880E09EE40197F1F7289A00C0289893
:100A000080E091E0FC013197F1F7289A00C0289826
:100A1000FC013197F1F75C98289A00C0289801975B
:100A2000F1F788E25EDF88E05CDFA1DF86E059DF76
:100A3000812F57DF1F910895991B79E004C0991FFA
:100A4000961708F0961B881F7A95C9F78095089528
:100A5000AA1BBB1B51E107C0AA1FBB1FA617B707E4
:100A600010F0A61BB70B881F991F5A95A9F7809500
:100A70009095BC01CD010895A1E21A2EAA1BBB1BC3
:100A8000FD010DC0AA1FBB1FEE1FFF1FA217B3075A
:100A9000E407F50720F0A21BB30BE40BF50B661F70
:100AA000771F881F991F1A9469F760957095809534
:100AB00090959B01AC01BD01CF010895FB01DC01C4
:100AC0008D91059080190110D9F3990B0895F89430
:020AD000FFCF56
:100AD2004465627567446973706C61792076310090
:0C0AE20020202020627920546F706900F1
:00000001FF
